:10029300010901011C19010800110A3F065B4F66A1
:0C02A3006D7D077F6F777C395E7971807C
:0B02D100EF1FAC0670011E4C70F622FF
:10023800C294C295D296D295C295D296D295C295BD
:10024800C296D295C295D296D295C2957F08E51BE3
:1002580025E0F51BC295D295309603431B01D29633
:08026800DFECD294AF1B7E0015
:01027000226B
:1002C100D2AF758901D2A9758C9E758A58D28C22BC
:1001F300AD07C2B1C2B075A0FFED75F00A1202716E
:10020300FF240AF8E6F4F5A0EF6002D2B07FE87E9F
:10021300031202D175A0FFC2B1C2B0ED75F00A128C
:100223000271AFF0740A2FF8E6F4F5A0D2B17FE8BB
:050233007E030202D170
:1002B0008F26E5096007AF261201F380F575090165
:0102C000221B
:10013000751C0FA2B2E433F51FA2B3E433F520A27D
:10014000B4E433F521A2B7E433F522A2B6E433F5E3
:1001500023A2B5E433F524D2B2C2B3C2B4D2B7C23B
:10016000B6C2B5851C1DD3E51D648094804015750D
:100170001E3CAF1E151EEF6007AF1D1201F380F28B
:10018000151D80E2E51F24FF92B2E52024FF92B303
:10019000E52124FF92B4E52224FF92B7E52324FF52
:0801A00092B6E52424FF92B59C
:0101A8002234
:10000E001202C1751C19D2B2C2B3C2B4C2B7C2B603
:10001E00D2B5851C25D3E525648094804009AF2593
:10002E001202B0152580EED2B2C2B3C2B4C2B7D29C
:10003E00B6C2B5751C05851C25D3E5256480948054
:10004E004009AF251202B0152580EEC2B2C2B3D25E
:10005E00B4D2B7C2B6C2B5751C19851C25D3E52519
:10006E00648094804009AF251202B0152580EEC23F
:10007E00B2D2B3C2B4D2B7C2B6C2B5751C05851C16
:10008E0025D3E525648094805003020011AF25121C
:06009E0002B0152580EB05
:03000B000201A946
:1001A900C0E0C0F0C083C082C0D075D000758C9EFD
:1001B900758A580508E508B40A14120238D3EF9471
:1001C90099EE648094804004C2978002D297E50832
:1001D900B42806750900750800209003120130D073
:0A01E900D0D082D083D0F0D0E032F5
:030000000200A457
:0C00A400787FE4F6D8FD7581260200EBA1
:10027100C2D530F707B2D563F0FF05F030E70CB215
:10028100D5F4048463F0FF05F080018430D502F4D5
:02029100042245
:1000B00002000EE493A3F8E493A34003F68001F258
:1000C00008DFF48029E493A3F85407240CC8C33351
:1000D000C4540F4420C8834004F456800146F6DF20
:1000E000E4800B0102040810204080900293E47E1B
:1000F000019360BCA3FF543F30E509541FFEE49315
:10010000A360010ECF54C025E060A840B8E493A3DB
:10011000FAE493A3F8E493A3C8C582C8CAC583CA06
:10012000F0A3C8C582C8CAC583CADFE9DEE780BEBE
:0102AF00004E
:00000001FF
